:100000009EC033C2B7C0B6C0B5C0B4C0B3C0B2C0E2
:10001000B1C0B0C0AFC0AEC0ADC0ACC0ABC0AAC074
:10002000A9C0A8C0A7C0A6C0A5C0A4C0A3C0A2C0A4
:10003000A1C0A0C0CAC9A1C8C3C99FC89EC8C8C919
:1000400041C99BC89AC891C971C997C8A1C916C9A5
:100050002DC993C892C891C825C938C9ECC88DC8A4
:100060008CC8DDC88AC889C888C887C886C885C8BA
:1000700084C883C882C881C8A6C87FC87EC87DC816
:100080007CC87BC87AC89CC886C877C876C880C830
:1000900074C873C872C871C870C873C816034700A3
:1000A00049004E004700450052002D004100560017
:1000B000520024036B00750077006100740061003A
:1000C000790040006E0069006600740079002E001F
:1000D00063006F006D00040309040902430002017C
:1000E0000080320904000001020201000524001012
:1000F000010424020205240600010524010301076E
:1001000005830308000209040100020A0000000739
:10011000050102010000070581020800001201012B
:100120000102000008C016E1050001010200014BB8
:100130004F4E46494755524154494F4E5F00112496
:100140001FBECFEFD4E0DEBFCDBF12E0A0E0B1E034
:10015000EEE6FAE102C005900D92A03FB107D9F793
:1001600014E0A0EFB2E001C01D92A031B107E1F7A9
:10017000F4DB7CCC45CFCF93DC01C62F809101010D
:1001800084FF0FC02091630398E82927209363031D
:10019000E4E6F3E09C2F02C04D9141939150E0F7CB
:1001A00004C03AE530930101F3CF6C2F84E693E06D
:1001B00058D1CC5FC0930101CF910895CF93DC015A
:1001C000C62F8091000184FF0FC02091580398E84A
:1001D000292720935803E9E5F3E09C2F02C04D91B5
:1001E00041939150E0F704C03AE530930001F3CF1A
:1001F0006C2F89E593E035D1CC5FC0930001CF919E
:1002000008951F93CF93DF9360917303161634F50F
:1002100080917003C3E8D3E0C81BD109635020E08C
:1002200010E880916F03803188F08D3209F44FC05F
:10023000B091F002B7FD50C0CE012FDA2FEF821738
:1002400009F44FC0811120E010E046C0CE0135DA3C
:1002500020917303121614F410927303C0910201DB
:10026000C4FF25C0809103018F3F09F1682F8930B9
:1002700060F5861B809303011BE48091F00280FDF2
:1002800013EC8F5F8093F002AEE4B3E087FD3BC0D8
:100290006623A1F560E070E0C62F693038F19EE179
:1002A000EFEFE093030110934D03909302019AE066
:1002B000F9B1F57011F49150D9F7992309F0A8C05C
:1002C0009093740390936E03A3C068E0D2CF3AE595
:1002D00030930201683089F11093F00220930301FA
:1002E000B7CF1EE11093020110E0F6CF8EE493E049
:1002F000B8D09C2F9C5FC830B0F6D2CFCD01BAD910
:10030000682F7727C9CFE0917103F091720386FFC0
:100310000DC0962F03C084918D9331969150D8F7DC
:10032000F0937203E09371037727B6CF962F02C044
:1003300031913D939150E0F7F3CF4881407651F5EC
:1003400046E553E0209356038981882389F420935E
:10035000570322E05093720340937103AF81AA23A5
:1003600009F0BACF8E81821708F0B6CF282FB4CF0C
:100370008530E9F08630F9F0883081F18930A1F1DB
:100380008A3081F18B3051F773EC70936303709373
:100390005803E4CFCE0146D9282F8F3FF9F6988134
:1003A00097FD02C01F7798CF2E811F7795CF5A8176
:1003B00050937403D3CF10EC8B818130C9F082301D
:1003C000B9F0833059F68A818823A9F424E086EDB8
:1003D00090E09093720380937103C0CF21E086E791
:1003E00093E0F7CF21E0B6CF6A8160937603B6CF72
:1003F000CE01D1D4D1CF813039F0823009F0AECFE7
:1004000026E18CE990E0E5CF24E282EB90E0E1CFB9
:10041000DF91CF911F91089520916900236020936F
:100420006900E89A83EC80936303809358030895EE
:10043000A82FB92F8FEF9FEF41E050EA615070F085
:100440002D9138E0722F782796958795269570FF25
:1004500002C0842795273A95A9F7F0CF809590950B
:100460000895E6DF8D939D930895CF93CFB7CF93F3
:10047000489BFECF489B09C0489B07C0489B05C0CE
:10048000489B03C0489B01C0A6C0DF93C091700386
:10049000DD27C958DC4F489B02C0DF91EBCF2F937B
:1004A0000F931F9309B12FEF00FB20F94F933F9358
:1004B00019B14FEF012700FB21F93BE031C04E7F1E
:1004C000012F19B1216028C0102F4D7F226000003C
:1004D00009B129C04B7F2460012F000019B12BC046
:1004E00019B1477F28602AC04F7E09B120612CC016
:1004F0004F7D19B120622FC04F7B09B1206432C0FB
:10050000422709B149934FEF0000102710FB20F953
:1005100019B11570C9F1297F91F2012700FB21F96A
:1005200009B1237F89F2315058F1102710FB22F9CD
:1005300019B1277E79F2012700FB23F92F7C81F284
:1005400009B1102710FB24F92F7971F200C019B1FD
:10055000012700FB25F92F7359F200C009B11027BC
:1005600010FB26F9223040F200C019B1012700FB30
:1005700027F9243028F64F77206819B10000F9CF09
:1005800011E01CBB00271CC03B503195C31BD04061
:1005900011E01CBB0881033C11F10B3401F12091E7
:1005A0006E031981110F1213EDCF4A81441F0936D2
:1005B00059F10D3211F0013E29F74F7009F0042F67
:1005C000009375033F914F911F910F912F91DF91F0
:1005D000CCB3C0FD4DCFCF91CFBFCF911895009137
:1005E0007503002379F3109173031123F9F5343067
:1005F000FAF13093730300936F03109170033BE0A3
:10060000311B3093700334C000917303013074F5D3
:100610000AE54F7049F43091020134FD2BC000937C
:100620000201CDE4D3E02AC0433049F0309101010A
:1006300034FD20C000930101C3E6D3E01FC0309118
:10064000000134FD17C000930001C8E5D3E016C0D7
:10065000052710E00BB91FC0052722C0052727C0BA
:1006600005272CC0052710E00BB933C04AE503C0AD
:1006700042ED01C0432FC4E1D0E032E01AB1156071
:10068000589A0BB11AB95F9355E020E820FF05276F
:100690000BB9279517951C3FD8F620FF05272795FE
:1006A0000BB917951C3FC0F620FF05272795179516
:1006B0000BB91C3F98F620FF0527279517951C3F7F
:1006C0000BB970F600C0499120FF05270BB927959B
:1006D00017951C3F38F620FF052727950BB917956E
:1006E0001C3F40F520FF0527279517950BB91C3FA8
:1006F00018F520FF0527279517951C3F0BB9F0F437
:10070000242F3A9519F60A7F5F910BB900001091DA
:100710007403110FC651D04011F010936E0311E015
:100720001CBB01601AB11A7F402F4A7F0BB91AB95E
:100730004BB948CF0527D2CF0527D7CF0527DCCF28
:100740008093F302282F3327F901EE0FFF1FEE0FDE
:10075000FF1FE20FF31FE20FF31FE758FD4F9081D9
:10076000909544B1492344B9B4B18181B82BB4B94F
:1007700075B1A0817A2B75B96281609557B1562306
:1007800057B947B19381492B47B9B8B18281B82B8A
:10079000B8B9A481A0957AB17A237AB95AB16581A2
:1007A000562B5AB94BB19481492B4BB9F901E05FF3
:1007B000FE4F80818430A0F063EA64BD53E055BDF4
:1007C00017BC18BC21EA209380003BE030938100E5
:1007D000109289001092880010928B0010928A006B
:1007E0007081763050F0E3EAE093B000F3E0F093EC
:1007F000B1001092B3001092B4000895482F1092E7
:10080000CD0310920F0410920E04282F3327F90104
:10081000EE0FFF1FEE0FFF1FE20FF31FE20FF31F9C
:10082000E758FD4F9081909574B1792374B954B114
:100830006181562B54B9B5B18081B82BB5B9A2816D
:10084000A09577B17A2377B967B19381692B67B99E
:1008500088B15281852B88B9B481B095AAB1AB23F8
:10086000AAB96AB17581672B6AB95BB19481592BBA
:100870005BB9F901E05FFE4F80818430A0F0B3EAFC
:10088000B4BDA3E0A5BD17BC18BC21EA209380002D
:100890003BE0309381001092890010928800109202
:1008A0008B0010928A008081863050F0E3EAE0935A
:1008B000B000F3E0F093B1001092B3001092B400D6
:1008C0004093F3021092F4021092F2020895FC0198
:1008D0008191DF018823A1F0E091CD0320910E04E6
:1008E000EF5F9E2F9F73E150921739F0FF27E35778
:1008F000FC4F8083E92F9093CD038D91882381F75E
:100900000895CF93DF93CDB7DEB723970FB6F89452
:10091000DEBF0FBECDBF9091F302E92FFF27EE0F90
:10092000FF1FEE0FFF1FEE0FFF1FEA5DFE4F22813C
:1009300033819927FC01EE0FFF1FE80FF91FDE013D
:100940001196E20FF31F83E001900D928150E1F7C1
:10095000662381F4E981FA8181E090E00B8002C096
:10096000880F991F0A94E2F7382F309580818323EE
:1009700080830DC0E981FA8181E090E00B8002C0A4
:10098000880F991F0A94E2F74081482B40832396F1
:100990000FB6F894DEBF0FBECDBFDF91CF910895A3
:1009A000EF92FF921F93CF93DF93CDB7DEB72397DC
:1009B0000FB6F894DEBF0FBECDBFAC018091F3023D
:1009C000E82FFF27E259FD4F708160E0671708F0BC
:1009D00048C07E010894E11CF11C142F1170E82F0F
:1009E000FF27EE0FFF1FEE0FFF1FEE0FFF1FEA5D49
:1009F000FE4F22813381862F9927DC01AA0FBB1F6E
:100A0000A80FB91FF701A20FB31F83E00D90019249
:100A10008150E1F71123B9F4E981FA8181E090E096
:100A20000B8002C0880F991F0A94E2F7982F9095C7
:100A3000108119231083569547956F5F671788F4C7
:100A40008091F302CACFE981FA8181E090E00B80C6
:100A500002C0880F991F0A94E2F73081382B308347
:100A6000EACF23960FB6F894DEBF0FBECDBFDF915D
:100A7000CF911F91FF90EF900895CF93DF93CDB763
:100A8000DEB723970FB6F894DEBF0FBECDBF9091AF
:100A9000F302E92FFF27EE0FFF1FEE0FFF1FEE0FF0
:100AA000FF1FEA5DFE4F208131819927FC01EE0F87
:100AB000FF1FE80FF91FDE011196E20FF31F83E01D
:100AC00001900D928150E1F7E981FA814081242F54
:100AD00033276B81462F552781E090E0042E02C01A
:100AE000880F991F0A94E2F72823392302C035950D
:100AF00027954A95E2F7822F992723960FB6F89407
:100B0000DEBF0FBECDBFDF91CF910895EF92FF9270
:100B10000F931F93CF93DF93CDB7DEB723970FB615
:100B2000F894DEBF0FBECDBF80E090E02091F302CD
:100B3000E22FFF27EB5FFE4F608161500AF442C055
:100B40007E010894E11CF11C8C01000F111FE22FA3
:100B5000FF27EE0FFF1FEE0FFF1FEE0FFF1FEA5DD7
:100B6000FE4F20813181862F9927DC01AA0FBB1F00
:100B7000A80FB91FF701A20FB31F83E00D900192D8
:100B80008150E1F7E981FA814081242F33277B816D
:100B9000472F5527A1E0B0E0042E02C0AA0FBB1FCB
:100BA0000A94E2F72A233B2302C0359527954A95FC
:100BB000E2F7020F111DC801615067FD03C02091CB
:100BC000F302C2CF23960FB6F894DEBF0FBECDBF9F
:100BD000DF91CF911F910F91FF90EF900895CF93E8
:100BE000DF93CDB7DEB723970FB6F894DEBF0FBE05
:100BF000CDBF9091F302E92FFF27EE0FFF1FEE0FFD
:100C0000FF1FEE0FFF1FEA5DFE4F268137819927F8
:100C1000FC01EE0FFF1FE80FF91FDE011196E20F36
:100C2000F31F83E001900D928150E1F7E981FA8191
:100C3000608323960FB6F894DEBF0FBECDBFDF9161
:100C4000CF910895AF92BF92DF92EF92FF920F93F0
:100C50001F93CF93DF93CDB7DEB723970FB6F894EA
:100C6000DEBF0FBECDBF8C01A090F302EA2DFF279F
:100C7000E05FFE4F8081DD24E82EFF24E114F104C3
:100C800089F15E010894A11CB11CC80139D1482F1B
:100C90003091F302E32FFF27EE0FFF1FEE0FFF1F30
:100CA000EE0FFF1FEA5DFE4F268137816D2D7727FE
:100CB000FB01EE0FFF1FE60FF71FD501E20FF31F39
:100CC00083E001900D928150E1F7E981FA81408340
:100CD0000E5F1F4FD3944D2D552747FD50954E1550
:100CE0005F059CF223960FB6F894DEBF0FBECDBF12
:100CF000DF91CF911F910F91FF90EF90DF90BF9008
:100D0000AF90089583B199278071907095958795DC
:100D10009595879595958795959587952091F50259
:100D2000222329F4813061F080E090E008952130A1
:100D3000D9F78823C9F78093F50281E090E0089500
:100D40008093F50282E090E008958091F302EBE158
:100D5000F1E0E80FF11D8081992708958091F30259
:100D6000E0E1F1E0E80FF11D80819927089580917D
:100D7000F302E5E0F1E0E80FF11D80819927089585
:100D800020E0281738F490E09E5C9A3FE8F32F5F4C
:100D90002817C8F30895FC018381813049F04AED9A
:100DA00050E0509372034093710383E490E0089500
:100DB0002DE131E0309372032093710382E190E0E2
:100DC000089590E0E92FFF27EE0FFF1FEE0FFF1FA2
:100DD000EE0FFF1FEE5FFC4F86E01192815087FF00
:100DE000FCCF9F5F973070F30895382F232F229503
:100DF0002F70FB01AB014F5F5F4F2A3060F4822FF1
:100E0000805D8083832F8F70FA01DA0111968A301A
:100E100060F4805D0BC0822F895C8083832F8F708C
:100E2000FA01DA0111968A30A0F3895C80831C9262
:100E3000CD010895CF93DF93EC01FB018D2F99270E
:100E4000282F22952F70AB014F5F5F4F2A30E8F4B7
:100E5000205D20838F70FA01DA0111968A30E8F460
:100E6000805D80838C2F2C2F22952F70AD014F5FDA
:100E70005F4F2A30E8F4205D2C938F70FA01DA017D
:100E800011968A30E8F4805D1CC0295C20838F7045
:100E9000FA01DA0111968A3018F3895C80838C2F6D
:100EA0002C2F22952F70AD014F5F5F4F2A3018F322
:100EB000295C2C938F70FA01DA0111968A3018F3AD
:100EC000895C80831C92CD01DF91CF910895982F8A
:100ED00080538A3010F499270895892F81548630E1
:100EE00040F0292F2156263040F49755892F992715
:100EF00008959753892F992708958FEF90E00895CB
:100F0000FC019081892F80538A3080F49927282F03
:100F1000332722953295307F3227207F32279181E7
:100F2000892F80538A30B0F4992731C0892F81549A
:100F3000863000F59753892F9927282F332722953C
:100F40003295307F3227207F32279181892F80533D
:100F50008A3050F3392F3154363020F49753892F8B
:100F6000992715C0492F4156463078F49755892F57
:100F700099270DC0292F2156263020F49755892F07
:100F80009927DBCF8FEF90E0C2CF8FEF90E0820FF9
:100F900099270895FC019081892F80538A3060F54C
:100FA0009927282F332722953295307F3227207FAB
:100FB00032279181892F80538A3098F59927820FA3
:100FC0009927782F6627DF0112962281822F80537E
:100FD0008A30C8F59927482F552742955295507F5A
:100FE0005427407F5427FD012181822F80538A306E
:100FF00090F5282F332761C0892F8154863008F05F
:1010000048C09753892F9927282F33272295329547
:10101000307F3227207F32279181892F80538A3079
:1010200068F2392F31543630E8F49753892F9927D5
:10103000820F9927782F6627DF0112962281822F4F
:1010400080538A3038F2522F5154563098F4275337
:10105000822F9927C0CFA22FA154A63098F42753EE
:1010600033272BC0492F4156463020F59755892FFD
:101070009927DECF922F91569630C8F42755822FAC
:101080009927A9CFB22FB156B63070F42755332720
:1010900014C0292F2156263020F49755892F9927DF
:1010A000B3CF8FEF90E07DCF2FEF30E006C08FEF12
:1010B00090E091CF8FEF90E082CFF42FF20F6F0F7F
:1010C000711DCB010895CF93DF93EC014EE050E00A
:1010D0006FE271E0BDD4892B69F48E85803328F0EE
:1010E0008A3318F4805399270BC0883539F080E093
:1010F00090E006C08BEB92E0EADBF9CF8AE090E06B
:10110000DF91CF910895FC018181803329F08133F3
:1011100041F080E090E008951092F40281E090E0C8
:10112000089581E08093F40281E090E00895FC014D
:101130008181803329F0813341F080E090E008958F
:101140001092F10281E090E0089581E08093F10235
:1011500081E090E00895FF920F931F93CF93DF9368
:10116000EC0188819927AA27BB27CF978433910563
:1011700020F4FC01E65EFF4F09948BEB92E0A7DBC5
:101180004BC211E01093F20210924203CE01F7CF4E
:101190002D98CE01F4CFD9DD882379F383E08093B5
:1011A000F202109242038EEB92E091DB77E87093AB
:1011B0007A001092040160E460937C0082E0C9C070
:1011C0002D9ACE01DCCF9981892F80538A3008F087
:1011D0004FC19927F82EFE0132969A81892F8053AC
:1011E0008A3008F03CC19927282F33272295329561
:1011F000307F3227207F32279181892F80538A3098
:1012000008F047C19927820F082F1127A7DDF8168C
:1012100008F0B3CF602F8F2DE2DCCE01B0CF8981F3
:10122000803309F480C1813309F0A7CF81E0809336
:10123000F402CE01A4CF9981892F80538A3008F01F
:101240003AC1C82FDD271C2FCF3F09F496CF7DDD93
:10125000C81708F092CF44E04093F2021092420384
:1012600080EC92E034DB37E830937A00C0930401DD
:101270001770106410937C0082E06BC09981892FF5
:1012800080538A3008F00EC1082F1127003108F072
:1012900074CF6DDD081708F070CF60E0802F31DB70
:1012A000CE016DCF80E0AADACE0169CF898180338B
:1012B00009F43DC1813309F060CFB1E0B093F10290
:1012C000CE015DCF31E030934203A6C1C2E5C093A9
:1012D00043031CDCAC01892F9927282F22952F70FE
:1012E0002A3008F0D4C0205D209344038F708A30E8
:1012F00008F0CBC0805D80934503842F242F229576
:101300002F702A3008F0BFC0205D209346038F70F5
:101310008A3008F0B6C0805D809347030AE20093EC
:1013200048031092490383E493E029CF0EDD88231C
:1013300009F423CFC2E0C093F20282EC92E0C7DA54
:1013400027E820937A001092040190E490937C00A7
:101350008C2F16DDA0917A00A061A0937A005091A5
:101360007A00506450937A0057C19981892F805335
:101370008A3008F0A9C0082F1127003108F0FDCEEF
:10138000F6DC081708F0F9CE61E0802FBADA88CFD2
:101390004EE050E06FE271E0CE015AD3892B09F0A4
:1013A000BCC08E85803308F452C08A3308F04FC029
:1013B00080539927882309F4E0CEC2D9CE01DFCE2D
:1013C000CE0101963FDCCE01DACE84EC92E0D7CE9E
:1013D000FE0131969981892F80538A3008F095C09B
:1013E0009927282F332722953295307F3227207F67
:1013F00032279181892F80538A3008F07EC0992747
:10140000820F9927782F6627DF0112962281822F7B
:1014100080538A3008F069C0282F3327422F552780
:1014200042955295507F5427407F5427FD012181DA
:10143000822F80538A3008F050C0282F3327F42F92
:10144000F20F6F0F711DCB01ABDACE0198CE88354C
:1014500019F080E090E0AECF8AE090E0ABCFA92F0A
:10146000A154A63008F070C09753892F9927BCCE9D
:10147000492F4154463008F0A9C09753892F992726
:10148000A9CE895C49CF295C40CF895C34CF295CE7
:101490002BCFE92FE154E63008F079C09753892F1C
:1014A0009927B1CE792F7154763008F07FC09753C9
:1014B000092F1127EBCE092F0154063008F056C032
:1014C0009753C92FDD27BFCE292F2154263008F08E
:1014D00075C09753092F112750CFA22FA154A630C2
:1014E00008F04DC027533327AACF522F51545630FE
:1014F00008F055C02753332791CF392F3154363058
:1015000060F59753892F99277BCF092F0154063017
:1015100090F49753892F992764CF8BEB92E0D7D91A
:1015200080E090E047CF1092F402CE0128CE1092D6
:10153000F102CE0124CE192F1156163008F04EC0FC
:101540009755892F99274DCFB92FB156B63008F04E
:101550004BC09755892F992747CE492F4156463082
:1015600008F04EC09755892F99274ACF192F115649
:10157000163008F03FC09755C92FDD2764CEB22F33
:10158000B156B63008F042C02755332758CFF92F4F
:10159000F156F63060F59755892F992734CE922F62
:1015A0009156963080F52755332738CF892F8156AD
:1015B000863018F59755092F112768CE692F615687
:1015C000663038F59755092F1127D7CE592F515628
:1015D000563038F49755892F9927FCCD8FEF90E03E
:1015E00000CF8FEF90E0F6CD8FEF90E0FDCD8FEF45
:1015F00090E009CECFEFD0E026CE0FEF10E046CE40
:101600008FEF90E0FDCE2FEF30E008CF2FEF30E0EE
:1016100016CF0FEF10E0B1CEDF91CF911F910F9158
:10162000FF900895FC012081822F99278076907089
:10163000809719F080E090E008959181392F305221
:10164000323098F0923241F027FDF4CF51E05093C0
:10165000000380E090E00895409101034423A1F746
:1016600022E0209301032081EFCF9093F8028FEFC7
:1016700090E008959C018091F802813219F080E099
:1016800090E00895F901A9EFB2E087E00D90019292
:101690008150E1F787E090E008959C018091F80285
:1016A000803241F4A9EFB2E0F90187E001900D9298
:1016B0008150E1F781E090E00895CF93DC01C62FDF
:1016C00020E0662309F190910F040FC01196903429
:1016D00050F4E92FFF27E253FC4F8083892F8F5F5F
:1016E00080930F04982FC15029F08C918A3271F7A2
:1016F00021E0ECCF213059F02FE3291B2930C0F431
:101700003FEF3093730314C090910F04F5CF9034E2
:1017100040F4E92FFF27E253FC4FC0839F5F909373
:101720000F048EEC93E017DDC0930F049C2FE4CFE1
:10173000CF9108950F931F93CF93E4DA99278130C7
:10174000910509F480C0029709F481C08091F202EA
:10175000882309F4FEC0813081F120917A0024FFB2
:10176000F8C0809178009091790097FDF2C095952E
:10177000879595958795982F82958F708A3008F078
:101780006CC0805D80934303892F8F708A3008F08E
:1017900062C0805D809344031092450383E493E02C
:1017A00096D8C091F202C43009F482C0C23009F464
:1017B00097C0C33009F0CDC052C080914203813040
:1017C00009F488C0A091F602B091F7021196B09387
:1017D000F702A093F6025F9709F0BBC002E70093FF
:1017E000430394D9AC01892F9927282F22952F7074
:1017F0002A3008F09AC0205D209344038F708A300D
:1018000008F091C0805D80934503842F242F22959A
:101810002F702A3008F085C0205D209346038F701A
:101820008A3008F07CC0805D809347031AE21093F1
:1018300048031092490383E493E049D81092F702D9
:101840001092F60286C081ED92E041D87FCF84ED00
:1018500092E03DD87BCF895C9DCF895C93CF70911E
:1018600004017F5F70930401072F112707FD109576
:101870006CDA9927081719070CF462C0909142039B
:10188000913009F446C010920401E0E4E0937C003A
:1018900082E076DAC0917A00C061C0937A00B0919C
:1018A0007A00B064B0937A0087ED92E010D851C00E
:1018B00030914203313069F18AED92E008D8A0916D
:1018C0007A00A061A0937A0080917A00806480936E
:1018D0007A003FC01092F2028DED92E0F8D739C045
:1018E000409104014F5F40930401042F112707FD2D
:1018F00010952BDA992708171907CCF01092F202ED
:101900005FEF5093040110927A0080EE92E0DFD7EF
:1019100020C01092F20282EE92E0D9D71AC0895C00
:1019200083CF295C7ACF895C6ECF295C65CF6091CB
:1019300004016770606460937C008C2F21DABFCF54
:10194000F0910401F770F064F0937C0082E018DA03
:10195000B6CFCF911F910F910895CFEFD4E0DEBFA6
:10196000CDBF48E150E03EE00FB6F894A895409313
:1019700060000FBE309360002AEF2BB985E08AB972
:10198000CFEF80E08150F1F7C150D9F7CAB944D503
:101990008C2F34D78C2FE82FFF27EE0FFF1FEE0F71
:1019A000FF1FEE0FFF1FEE5FFC4F96E0119291506C
:1019B00097FFFCCF8F5F873070F310920103109276
:1019C00000037894A8951DD4B5DE5091010154FF11
:1019D00024C020910E04422F552743575C4F80911D
:1019E000CD03821708F480E4821B282F3327C22FEF
:1019F000222321F460910003662379F0C83008F1B6
:101A0000C8E071E0709300036C2FCA01B4D39091C9
:101A10000E049C0F9F7390930E04909101039923E1
:101A200089F2A0910001A4FFCDCF923069F062E06D
:101A30008EEE92E0C3D3B0910103B150B093010395
:101A4000C1CF10920003E0CF68E086EE92E0F2CFC3
:101A5000FB01DC014150504030F08D910590801920
:0E1A600019F40020B9F7881B990B0895FFCFE9
:101A6E005A5A5AFFFF00040004001000000000083C
:101A7E000004040606000000000000000406040630
:101A8E0000000000000000000000000000006202E4
:101A9E0056024A023E023802560226023E026202F6
:101AAE0020024A020E023802200226020E02DE0137
:101ABE000000000000000000AE0100000000000069
:101ACE00AE01000000000000000000000000000059
:101ADE0000000000000096017E01000000002B00B7
:101AEE00062B00052500012500022500032B00030F
:101AFE002B00042B000726000026000126000226DC
:101B0E0000032600042600052300002900012800FA
:101B1E0000280001280002280003280004280005E0
:101B2E002500002B00012B00062B000525000125AA
:101B3E0000022500032B00032B00042B00072600B8
:101B4E0000260001260002260003260004260005BA
:101B5E002300002900012900062900052300012386
:101B6E00000223000329000329000429000747006F
:101B7E00004800008800008A0000B30000B4000096
:101B8E002B00042B00072800002800012800022843
:101B9E000003280004280005230000290001470047
:101BAE00004800008800008A00002800002800017C
:101BBE002800022800032500032B00032B00042B12
:101BCE00000726000426000523000029000100045A
:101BDE000400000010100000081F203F00FA001142
:101BEE002E3F0002F8112E3F0002F8112E3F000288
:101BFE00F8112E3F0002F81F203F00FA00102F00B0
:101C0E00FA00FA102F003F00FA1F203F00FA001FC3
:101C1E00203F00FA00112E3F0002F8212A00690031
:101C2E00530049003F312E302E302E306176722A0D
:101C3E00004E2A00462A002A69002A5300452A002F
:101C4E002A002A452A00A1200000000002000300FD
:00000001FF
